:020000040800F2
:1000000090080020C94C0008E54C0008E94C0008A5
:1000100000000000000000000000000000000000E0
:10002000000000000000000000000000ED4C00088F
:100030000000000000000000EF4C0008B548000878
:100040007F11000800000000971100084B12000803
:100050009F120008AF17000833180008371800086F
:10006000000000002F450008532D0008C33600088B
:100070001737000873380008E7390008000000004F
:10008000093900080000000000000000BB3B000828
:1000900000000000033300080D330008AF4A0008D9
:1000A00000000000D34A0008000000000B2E0008EA
:1000B000FDB5B2B03A98049102A93B2288540020C1
:1000C0000D9026A8401C31900DE00498329A90477C
:1000D0000490002801D100F037FF0D98401C0D90CE
:1000E0003398401C339033980178002910D025298B
:1000F000EBD100200790089009900A900B900C908B
:10010000002102240120139008201290339D05E065
:100110000D9800F01BFF0800139901436D1C28780F
:100120002028F8D023280BD02B2804D02D2804D049
:10013000302808D00AE02143F0E708000421ECE76A
:1001400008000821E9E708001021E6E72A280FD176
:10015000349802681068121D349B1A600F900028B2
:1001600004D542420F920800042101436D1C12E0A5
:1001700000200F90654A09E00F9B934205DA9E002C
:10018000F3185B00181830380F906D1C28780300A6
:10019000303B0A2BF0D328782E2803D00020C04310
:1001A0000E9027E06D1C28782A2808D13498006822
:1001B0000268001D349B18600E926D1C1AE02D28F9
:1001C00002D12D226D1C00E0002200200E900CE0D8
:1001D000002A09D10E9B4D4EB34205DA9E00F3185A
:1001E0005B00181830380E906D1C28780300303BE7
:1001F0000A2BEDD302A801872E78310041487844BC
:10020000FF30C01C00F086FF002801D06D1C00E00C
:10021000002602A83A214654405C682804D1287878
:1002200068280BD1622005E06C2807D128786C285B
:1002300004D1712002A93A2288546D1C17A8069097
:10024000287869460870681C33906846057828004D
:10025000253833D01C3800D10EE2001F022800D808
:100260000AE2133801D100F093FD093800D103E20E
:10027000801E01D100F029FE401E01D100F0D6FD04
:10028000401E022800D8F7E1001F01D100F0CEFD8A
:10029000401F00D149E1401E01D100F079FD401E10
:1002A00000D1EBE0C01E10D0801E01D100F070FD27
:1002B000C01E01D100F06CFD00F012FE252017A930
:1002C00008701398079000F016FE349800680468D0
:1002D000001D349908600594002C00D0BAE002A8F3
:1002E0003B21405C002800D1ADE00024E4430648F7
:1002F0007844143000F018FF201A01D000F024FEDA
:1003000000F0F9FDFC47000030480000CBCCCC0CDD
:10031000641E01D000F00EFE3295079D17AC002D33
:100320000FD0329E227802A9300000F0C7FE0028CC
:1003300002D4641C6D1EF5D13296002801D000F065
:1003400003FE3020694608700A9C002C0DDD329DAA
:1003500001236A4602A9280000F0C1FE002801D04E
:1003600000F0F2FD641EF3D13295059C089D002D2E
:100370000FD0329E227802A9300000F09FFE0028A4
:1003800002D4641C6D1EF5D13296002801D000F015
:10039000DBFD302769460F700B9C002C0DDD329D74
:1003A00001236A4602A9280000F099FE002801D026
:1003B00000F0CAFD641EF3D13295059808994418DF
:1003C000099D002D0FD0329E227802A9300000F046
:1003D00075FE002802D4641C6D1EF5D132960028EB
:1003E00001D000F0B1FD684607700C9C002C0DDDBB
:1003F000329D01236A4602A9280000F070FE002801
:1004000001D000F0A1FD641EF3D1329502A838217D
:10041000405C400700D466E62020694608700198D9
:10042000002800DC5FE6019C329D01236A4602A998
:10043000280000F054FE002801D000F085FD641E65
:10044000F3D132954FE63F487844FF30C01F059006
:1004500000F051FD0E9D002D03D5200000F088FE18
:1004600009E02A000021200000F08AFE002801D0C7
:10047000001B00E02800089000F03DFD3498006863
:100480000268001D349908600020C043002110401C
:1004900002AA03C217A80590069A3C2302A803C823
:1004A000002904D1002802D10E9C002C13D05B1E21
:1004B00005072D0F3035EEB23A2E00DB2735D55427
:1004C00000090C072043090901D1002803D0059C2D
:1004D000D518AC42EBD33C20C01A0890D118059136
:1004E0000E99884208DA081A0A9002A8018FBC4ABD
:1004F0000A40028700F0FFFC002901D400F0FBFC59
:1005000002A93822895C14220A40102A01D000F086
:10051000F2FC0F99079A891A0A9A891A081A002870
:1005200001DC00F0E8FC00F031FC02A83B21415C5A
:10053000002909D00024E4434B487844FF302B3095
:10054000D8E600BF104600003A21405C62286AD01D
:10055000682819D06A2845D06C2806D071284FD059
:10056000742831D07A2821D06FE03498006801686F
:10057000001D349A106000297AD10024E4433B48DE
:100580007844FF301738B5E6349800680168001DDC
:10059000349A1060002905D10024E443334878449C
:1005A000CA30A7E60D98088000F0A5FC34980068D2
:1005B0000168001D349A1060002959D10024E443D9
:1005C0002A487844A63095E6349800680168001DF2
:1005D000349A106000294BD10024E4432348784426
:1005E0008A3087E6349800680268001D34990860F4
:1005F000002A13D10024E4431C4878446E3079E685
:10060000349800680268001D34990860002A05D1FA
:100610000024E4431548784452306BE60D98C11726
:1006200003C200F068FC349800680168001D349A29
:100630001060002905D10024E4430C4878442C3094
:1006400058E60D98087000F056FC34980068016870
:10065000001D349A106000290AD10024E4430348A5
:100660007844083046E600BFA0440000B4440000CF
:100670000D98086000F03FFC34980268D21D0720F6
:1006800082433498026003CA349B1A6002AA03C2F0
:100690002022C80F04D007982D2117AA11540DE06D
:1006A00002A8008F204204D007982B2117AA1154CA
:1006B00004E0C00704D5079817A90A54401C079006
:1006C00017A807994318059326AA02A803C814ACD3
:1006D00003C468460078202101436846817061297F
:1006E00009D00E98002801D5062003E003D1672920
:1006F00001D113980E9002A803C8080041004915C3
:10070000491C10D100030ED003200890613D1A2D22
:1007100004D250497944FF313D3116E04E497944C5
:10072000FF31373111E002A803C808004100491524
:10073000491C0FD100030DD103200890613D1A2DF3
:1007400015D346497944FF3115310322180000F0D2
:100750003DFDD0E302A830C8B9A003C82940002657
:1007600080277F03B94207D2002069400DE03C4951
:100770007944FF311339E8E7080DAF4E36182000F1
:100780002900B14D0D40AD49294302AB03C3684672
:10079000807861280FD1059830210170811C059166
:1007A00069460978612901D1782100E0582141701A
:1007B0000798801C079002A803C8A1A430CC04406D
:1007C0000D4002D1002C00D181E16846807861287B
:1007D00000D0BCE00E98002804D5212003E000BF23
:1007E000EFFF0000401C1690169F7F1C14A803C842
:1007F0000022002300F0F7FC02A830C802D28020BB
:1008000000064540361F019626A90A7026A8461CF8
:10081000002F54DD20002900002280235B0300F01C
:10082000FBFC4CD869004A0D11001C31002A19D07C
:10083000002917DDB24A914206DB1005290080220B
:1008400012061140014311E07F4A2A400805104377
:1008500005000DE0044300000443000008430000CD
:1008600000430000290080221206114000240D00E0
:100870002000290000F0EAFC1490FF1F002F09DD82
:1008800000F01EFD02000B002000290000F085FD95
:1008900004000D00F01D0721149A002A0ADD491EEC
:1008A00008D4401E13071B0F03701211F5E7401EFA
:1008B00000220270491EFAD5C61D002FAADC26A808
:1008C0003199711A26AA521C169B0C00994200DD20
:1008D0001C00002C34D48C4205DA411C095D082927
:1008E00001DB0F2100E00021230026ADED1801E01F
:1008F000641E6D1E5B1E2E788E42F9D00F2904D126
:10090000411CC95C491C401CC154002B04D526AABB
:10091000641C0198001D0190611E11D45318684693
:1009200000781D783035EEB23A2E02DB06003A3EF2
:10093000AD191D70491E5B1E0029F2D5694608706D
:100940000E98002800D4C1E0601E0E90BEE014A8EE
:1009500030C86D006D086C49300048436B4900F0A9
:10096000A9FD019007200199401A05DD0200200031
:10097000290000F07DFB0AE042420020644900F0BB
:1009800077FB02000B002000290000F0EDFD6A4615
:100990009278662A02D1019A0A3200E006220E9B62
:1009A0009A18142A00DD142226AB30241C705C1C1B
:1009B00002E014A803C8169A002A47DD14AB03C34B
:1009C000169214A803C800F053FC30900646083471
:1009D000042530000A2100F070FD0F0030000A21CC
:1009E00000F06BFD06003037601E077030000A21F2
:1009F00000F063FD0F0030000A2100F05EFD0600EC
:100A0000A41E303727706D1EE3D1083416980838BD
:100A100016900028CDDD309800F042FC02000B005B
:100A200014A803C800F0B9FC00223A4B00F0FDFD09
:100A300014AA03C2C5E700BF02FCFFFF0000E03FAD
:100A4000FFFFFFFFFFFFFF7FFFFF0F803198201A9E
:100A500026A94A1C019902E0401E491E521C137827
:100A6000302BF9D0019169468978662902D1019924
:100A7000491C06E069468978652901D1139900E08F
:100A800000210E9B5C18A04200DA441E002C1DD4ED
:100A9000844204DA105D342801DD392100E0302180
:100AA0002300501EC51801E0641E6D1E5B1E2E78CB
:100AB0008E42F9D0392902D1D15C491CD154002B86
:100AC00004D50200641C0198401C0190019D160091
:100AD000684600786946487000F06AFE406A00780F
:100AE000694608700E9F20B2002803DC139C054E57
:100AF0007E4410366846807866280DD16D1C25E04E
:100B0000FF0700006440000097750000A086010008
:100B10000000F03F84D7974168468078672847D126
:100B200028B20321C943884248DBB84246DA6D1C2B
:100B300002A8008F1299C0B2084203D120B2B84275
:100B400000DA070028B23F1A00D5002728B2002893
:100B500000DDB7E00898411C08913021059A115436
:100B6000002F05DC02A8008F1299C0B2084206D0FF
:100B70000898411C089169460978059A115428B2D1
:100B800041428F4200DA7D422DB268420B907D19BE
:100B900020B2854200DA2C0024B2099422003100F0
:100BA0000598089BC01800F011FB281B0C90D7E09B
:100BB00068464078612818D170201BE020B2B84206
:100BC00006DA02A9098F129AC9B2114200D10700B0
:100BD0007F1E00D5002768464078672802D165202F
:100BE000694607E04520694604E0684640784128A8
:100BF00001D1502048700898411C08913178059A1D
:100C00001154711C002F05DC02A8008F129AC0B28B
:100C1000104219D00898421C08926A461278059B27
:100C20001A54002F10DD641E20B2874200DA3C0007
:100C300022B20598089BC01800F0C8FA24B20898A0
:100C400000190890381B0B900598089940186946C0
:100C50004978017029B2002903D42B214170861CE8
:100C600003E02D224270861C4D42002412A9280068
:100C70000D0005E00A2100F01DFC2970641C6D1CAC
:100C800000B20028F6DC012C08DC68464078202100
:100C90000143652902D130203070761C002C09D127
:100CA00030203070761C07E0641E12A8005D3030E2
:100CB0003070761C002CF7DC059808994018301A23
:100CC00009904DE020B229B288421EDA22B23100EA
:100CD0000598089BC01800F079FA24B2089800190A
:100CE00008902DB2291B0B91002F05DC02A9098F5A
:100CF000129AC9B2114206D069460978059A115470
:100D00000998401C09900C972AE02AB231000598F6
:100D1000089BC01800F05AFA28B2089909180891DF
:100D2000641B002F05DC02AA128F129BD2B21A425A
:100D300005D04A1C08926A461278059B5A5421B283
:100D40008F4200DA3C0022B231180598089BC01887
:100D500000F03CFA24B2089800190890381B0B9058
:100D600002A83821405C14210140102900D0C2E0C3
:100D70000798089940180B994018099940180C9940
:100D800040180F99884200DBB5E0081A0A90B2E0DB
:100D900002AA3A20105C622808D068280ED06A287F
:100DA00014D06C281DD0712810D01AE03498016836
:100DB0000868091D349B1960C0B218E034980168B6
:100DC0000868091D349B196080B210E034980368EC
:100DD000DB1D072083433498036003CB349C2360DE
:100DE00006E0349801680868091D349B19600021E9
:100DF00002AB03C3108F1299C0B208425BD002A8A5
:100E000003C8002901D1002855D068460078202168
:100E1000014378294FD1079817A930220A54401C62
:100E2000421C07926A4612780A5444E002AA3A2009
:100E3000105C622808D068280ED06A2814D06C286C
:100E40001DD0712810D01AE0349801680868091D77
:100E5000349B196040B218E0349801680868091D95
:100E6000349B196000B210E034980368DB1D072042
:100E700083433498036003CB349D2B6006E03498A1
:100E800001680868091D349B1960C11702AB03C3D0
:100E9000002902DA07982D2109E0108F204202D0A4
:100EA00007982B2103E0C00705D50798202117AA32
:100EB0001154401C079017A80799401805906846E0
:100EC000017802A800F044F815E0139807903498D0
:100ED00000680168001D349A106017A801700AE0CC
:100EE000252017A9087013980790684600780028F5
:100EF00001D04D7007940F980799401A0A99401A2B
:100F00000899401A0B99401A0999401A0C99401AED
:100F1000019002A83821405C400701D5FFF7FDF998
:100F20002020694608700198002801DCFFF7F5F9D8
:100F3000019C329D01236A4602A9280000F0CFF8E7
:100F4000002801D1FFF7E4F90020C04335B0F0BD1F
:100F5000F2B586B0040025696F2901D1082707E0A2
:100F6000084620210143782901D00A2700E01027F4
:100F70003C2603CC083C04AA03C26A46127E642ABB
:100F800003D06A46127E692A09D1002907DA04A82B
:100F900003C800220023121A8B4104A80CC004A825
:100FA00003C800290DD100280BD1206B002808D1DF
:100FB000082F3BD13820205C000737D53B26302056
:100FC00033E00294009504A830C8761E01962000F4
:100FD00029003A00FB1700F0F1FB3032D0B23A287A
:100FE00003DB6846007E51381218009882552000B5
:100FF00029003A00FB1700F0E1FB04000D0001D1CD
:10100000002C05D00298C068009989198842DCD369
:10101000029C009D082F09D13820205C000705D5CF
:10102000A85D302802D0761E3020A8553C20801BB9
:10103000A061A919E160216B884206DA081A2062D2
:10104000208F1C490140218710E000290ED538214E
:10105000615C14220A40102A08D1616B6269891A06
:10106000226A891A081A002800DD206207B0F0BD44
:10107000F8B50026104F04000D00009214E0C007E0
:1010800007D532003B002000290000F0CEFA040012
:101090000D000098401000903000390032003B00F5
:1010A00000F0C3FA06000F0000980028E7D12000E6
:1010B0002900F4BDEFFF00000000244010B503003C
:1010C0000C001100A0689847A060002804D0E06AD6
:1010D000401CE062002010BD0020C04310BDF8B5E8
:1010E0000024002B11D007000E0014001D002178F1
:1010F000B068B847B060002809D0F06A401CF062C0
:101100000020641C6D1EF2D104002000F2BD0020FE
:10111000C043F9E7C9B202788A4203D0401C002AD2
:10112000F9D1002070472E0080B5002801D100BF02
:1011300007A006490B68002B03D022220021984704
:1011400001E000F070FB222002BD000084040020BA
:10115000636F6E73747261696E742068616E646C23
:1011600065723A20626164206D6573736167650022
:10117000431C0178401C0942FBD1C01A7047FEE7AE
:10118000C9B2521E05D30378401C8B42F9D1401ED0
:10119000704700207047FEE770B4103A03D378C957
:1011A000103A78C0FBD2530701D318C918C001D533
:1011B00008C908C0D20704D30B880380891C801C8F
:1011C000002A01D50B78037070BC70478B0701D1E2
:1011D0008307E1D0124205D00B78491C0370401CF4
:1011E000521EF9D1704730B4012464054D00EC4221
:1011F0000BD85D00EC4208D80C001C43640004438B
:10120000144304D2994200D1904230BC7047FCD0C4
:101210008B42FAD18242F8E730B4012464054D00D4
:10122000EC420BD85D00EC4208D80C001C43640073
:101230000443144304D28B4200D1824230BC704735
:10124000FCD09942FAD19042F8E7FEE7F4464A18FA
:1012500005D200F00FF801D580174008604700F074
:1012600009F80121C907884200D9080040426047B7
:101270004A1812D2400DC90208430121C907084388
:10128000520D40210901521A521C06D452421F32FB
:1012900001D4D0407047C017704700207047FEE768
:1012A000010042221201D21E004207D002D4521E77
:1012B0000018FCD5C10A40051205891870470000C6
:1012C0000100EED54042F446FFF7EBFF0122D207C2
:1012D00011436047F0B40125ED070F005F404FD484
:1012E0008B4200D1824205D98446100062468C466A
:1012F00019006346DF184C18640D7F0D3AD0661C48
:10130000760537D0E61B352E34DCDB022B43DB0AB7
:101310000C0DC9022943C912202E0DDB1700203EF7
:1013200006D01F00F741F3405F400026012A7741B5
:10133000C01871410DD217E01700F741F240574035
:10134000F3415A40B340F3405A40002680185941B7
:101350000AD3A21C52050FD0C207012F72411700F9
:101360004008CB0718434908641C24054208AF41D4
:1013700070416141F0BC7047641C21050020F9E711
:101380006B4010E06B40ABE7F742F3D1E943F1E784
:101390002442EFD100200021ECE7F0B40125ED0755
:1013A0000F005F40EED40C00871A9C4105D2C01B91
:1013B000A141D219634169406B40AE0ADF184C1855
:1013C000F442E1D2640D7F0DE2D0E61B362ED1DC73
:1013D000DB022B43DB0AA4460C0DC9022943C90AD0
:1013E000012E28DC04D1D6075208DF073A435B08F8
:1013F000EF0A76429041994114D039423BD1B61957
:1014000040414941761C394204D1761C00184941BB
:101410003942FAD0B9436746B74208D9A41B24051C
:101420002143A7E70042EAD13642E8D1A2E7E40A25
:10143000E10700209EE7202E0BDD203E1F00F34039
:10144000F7415F40012A002257417E429841914175
:101450000BE01700F741F2405740F3415A40B340C8
:10146000F3405A407E42904199410A0303D2641EE0
:10147000B619404149410027641E24054208AE4187
:1014800078416141F0BC7047F446002804D44942D9
:1014900000F013F8404260474042002905D45FD075
:1014A00000F00BF8404249426047494200F005F81D
:1014B0004942604703460B43E6D40022030A8B42AD
:1014C0000BD203098B4219D243088B422ED2411A08
:1014D00000D20146524110467047FF2209023FD018
:1014E00012068B4205D3121209028B4201D312124B
:1014F000090203098B4219D300E0090AC3098B4290
:1015000001D3CB01C01A524183098B4201D38B0115
:10151000C01A524143098B4201D34B01C01A5241B8
:1015200003098B4201D30B01C01A5241C3088B42FD
:1015300001D3CB00C01A524183088B4201D38B00E8
:10154000C01A524143088B4201D34B00C01A52418A
:10155000884200D3401A5241CFD20146104670470C
:1015600008B500F065F908BDF0B40E005E40012535
:10157000ED072E40B446AE0ADF184C18F4423BD2B9
:10158000F74241D2640D43D07F0D38D0E41BC9022D
:10159000DB0229432B43CF0ADB0A0600B61A9F4120
:1015A00004D2641EB6197F41B6185F416812800DDF
:1015B00024180018844222DAE80C0021B6197F4171
:1015C000B61A9F4102D2B6185F413F1C40414941C3
:1015D000F4D3241C21DD2405B6197F41B61A9F419E
:1015E00005D33743C60737430026012F70416141B9
:1015F00066463143F0BC7047FCD1F74205D200206B
:10160000C14349054908F3E704D00020C143F1E78D
:101610007F0DFAD000206146ECE72442FAD1401C4D
:1016200061410F03F6D30020E2E7F0B50E005E4003
:101630000125ED072E40B446AE0ADF184C18F442DF
:1016400008D2F7420ED2640D01D07F0D12D10020D6
:101650006146F0BD05D1F74201D87F0D05D10020CC
:10166000C143F0BDFBD1640DF9D00020C143490551
:1016700049088FE0E419C902DB0229432B43DB0A46
:10168000460DC00231438E4630B487B295B27D43D9
:101690002E0CADB2140C7C43A419260C2404254353
:1016A0009CB27C43A419190C7943270CC919A4B224
:1016B0000F043C43090C000C97B247432E0CBE1993
:1016C0003543ADB2170C4743360CBF19A6B2BF194C
:1016D0003E043543240C3E0C36199FB24743BF19D4
:1016E000BCB23E0C89191F0C47437F183E0434439B
:1016F000390C704680B297B247432E0CBE19354361
:10170000ADB2170C4743360CBF19A6B2BF193E0441
:101710003543240C3E0C36199FB24743BF19BCB267
:101720003E0C89191F0C47437F183E043443390C83
:1017300077463F0C90B278432E0C80190604ADB268
:101740002E43050CA0B22D18120C7A435019020C2E
:1017500080B2240CA4189AB27A43121914042043BC
:10176000120C89181B0C7B43C91830BCEF0A394294
:1017700003D1B61940414941641E6F12BF0DE41BED
:101780000BDBFF19BC4211DA240500274208AE41E9
:101790007841614166463143F0BD641C05D1401C6F
:1017A0006141CF0201D34908F4E750E75DE7FEE766
:1017B000014870470000000058000020124224D069
:1017C000994228D970B500251B4202D00C00002197
:1017D00009E00024012649186441944200D3A41A68
:1017E0007641F8D33100012601E0764109D2001894
:1017F00064416D41A41A9D41F7D2A4185D41B61908
:10180000F5D3300022002B0070BD1B42D8D108B5A3
:1018100000F010F808BD01D19042D3D202000B00B5
:1018200000210020704780B5012000F005F801BDBF
:101830007047FEE77047FEE780B500BF00BF024A71
:1018400011001820ABBEFBE72600020010B5040013
:10185000002C01D1012035E0A0690028FFD1E06F04
:10186000002805D1002078216054200000F094FD6C
:101870002420E0672068006801218843216808600F
:10188000200000F0D9F9012801D101201AE0606A96
:10189000002802D0200000F089FA206840680A4938
:1018A00001402068416020688068082188432168E1
:1018B00088602068006801210143206801602000E1
:1018C00000F0ECFA10BD0000FFF7FFFF38B5040090
:1018D000002C01D101201BE02420E0672068006873
:1018E0000121884321680860002520680560206880
:1018F000456020688560200000F04FFD8420255061
:10190000E5678020255025666566782025540020EF
:1019100032BDFEB504002068C769206805682068EC
:1019200080680090BF4838400290029800280AD191
:10193000B80608D5A80606D5A06E002802D020005B
:10194000A16E88476BE10298002800D1A6E0012033
:1019500000990140002904D1B3492940002900D150
:101960009CE001003940C9B2002908D0E90506D53C
:10197000216808628421615801438422A150B9077B
:101980000DD500990140C9B2002908D00221226872
:1019900011628421615804220A438421625079072C
:1019A0000DD500990140C9B2002908D00421226850
:1019B00011628421615802220A438421625039074E
:1019C0000ED5A90604D400990840C0B2002807D05B
:1019D00008202168086284216158084384216050EE
:1019E00038050BD5680109D58020000121680862FF
:1019F0008420205820210143842021508420205815
:101A000000284AD0B80607D5A80605D5A06E00283C
:101A100002D02000A16E88478420205801904026E3
:101A2000206880683040002804D1019828210140B6
:101A300000292CD0200000F05FFB20688068064061
:101A4000002E20D0EFF31080012181F3108821684F
:101A50008968402291432268916080F31088606F0A
:101A600000280CD07148616F4863606F00F057FD2B
:101A7000002812D0606F616F496B88470DE020002D
:101A800000F00CFE09E0200000F008FE05E0200058
:101A900000F004FE002084216050C0E0206E012888
:101AA00000D0A9E0F80600D4A6E0E80600D4A3E040
:101AB0001020216808622068806840065AD5606F4F
:101AC00000684668300080B2002852D030005821AB
:101AD000615A80B288424CD25A202652606F806987
:101AE00020283BD0EFF31080012181F3108821687A
:101AF00009684F4A0A4021680A6080F31088EFF3B2
:101B00001080012181F310882168896801229143A6
:101B10002268916080F31088EFF31080012181F337
:101B2000108821688968402291432268916080F37F
:101B3000108820208021605000202066EFF3108064
:101B4000012181F3108821680968102291432268DD
:101B5000116080F31088606F00F0BBFC02206066AB
:101B60005820205A5A21615A411A89B2200000F0A7
:101B700096FD54E05820205A5A21615A461A5A209C
:101B8000205A002837D0300080B2002833D0EFF33D
:101B90001080012181F3108821680968254A0A40D4
:101BA00021680A6080F31088EFF31080012181F32F
:101BB000108821688968012291432268916080F32E
:101BC000108820208021605000202066A066EFF35E
:101BD0001080012181F31088216809681022914347
:101BE0002268116080F3108802206066310089B29B
:101BF000200000F054FD12E0380608D5280606D56E
:101C0000E06E002802D02000E16E884707E07806E9
:101C100005D5680603D5200000F0B4FAFFE7F7BD4C
:101C2000000000000F080000200100046D210008E2
:101C3000FFFEFFFFDFFEFFFFFEB5050000263000C0
:101C400069460870A868296901436A690A43E86916
:101C50001043296809688D4A0A40024329680A60CE
:101C6000296849688A4A0A40E96811432A6851602C
:101C7000A9692A6A0A43029229688968854A0A4042
:101C8000029911432A689160834909688907890F7D
:101C9000002905D0022909D006D3032902D007E084
:101CA000340006E0022404E0042402E0082400E0FA
:101CB000102480273F02E869B8423FD12000C0B21B
:101CC000002806D0022808D0042808D008280AD006
:101CD0000AE001F013F807000AE0A24F08E000F064
:101CE000DDFF070004E003E03700012069460870CB
:101CF000002F56D002207843696849084018696867
:101D0000FFF7DBFB01900198102813D30198802185
:101D1000490288420ED20199934808400199490826
:101D20004907490F01436846418068464088296851
:101D3000C86036E001206946087032E02000C0B279
:101D4000002806D0022808D0042808D008280AD085
:101D50000AE000F0D3FF07000AE0824F08E000F03D
:101D60009DFF070004E003E037000120694608708A
:101D7000002F16D06868400838186968FFF79DFB87
:101D800001900198102809D30198802149028842C6
:101D900004D2019880B22968C86002E00120694637
:101DA0000870AE66EE6668460078FEBD00B5242178
:101DB000415CC90707D5016849686C4A0A40816AD5
:101DC0001143026851602421415C890707D50168ED
:101DD0004968674A0A40C16A114302685160242178
:101DE000415C490707D501684968BB4A0A40016B55
:101DF0001143026851602421415C090707D501683D
:101E00004968B64A0A40416B114302685160242177
:101E1000415CC90607D501688968B14A0A40816BEF
:101E20001143026891602421415C890607D501684D
:101E30008968AC4A0A40C16B114302689160242151
:101E4000415C490614D501684968A74A0A40016CFB
:101E5000114302685160016C80225203914207D104
:101E600001684968A14A0A40416C11430268516007
:101E70002421415C090607D5016849689C4A0A404B
:101E8000816C11430268516000BD0000F369FFFFDF
:101E9000FFCFFFFFFFF4FFFF301002407CB50500CD
:101EA000002484202C5000F04DFF060028680068B4
:101EB00000071DD58F480090330000228021890340
:101EC000280000F057F8002812D0EFF3108001210D
:101ED00081F3108829680968802291432A6811607B
:101EE00080F310882020E86778202C54032038E005
:101EF0002868006840072BD57E48009033000022F8
:101F00008021C903280000F035F8002820D0EFF325
:101F10001080012181F31088296809688F4A0A40DE
:101F200029680A6080F31088EFF31080012181F3A3
:101F3000108829688968012291432A68916080F39A
:101F4000108820208021685078202C54032008E03D
:101F50002020E867802168502C666C6678202C541D
:101F6000002076BD00127A00F0FF0000FFFFFDFFA9
:101F7000FFFFFEFFFEB504000F00089D2068C0694A
:101F80003840B84201D1012000E0002069460979BB
:101F9000884237D10020C0438542EFD000F0D2FE06
:101FA0000299401A854201D3002D01D103202AE075
:101FB000206800684007E1D508262068C0693040E5
:101FC00000280BD020680662200000F095F88420DD
:101FD0002650002078216054012014E08020000168
:101FE0002168C96901400029C8D021680862200021
:101FF00000F082F820208421605000207821605475
:10200000032000E00020FEBD70B503005965582094
:102010001A525A201A5200249C66802040019D6862
:1020200085420AD11D69002D03D14D4D5C269D537B
:1020300014E0FF255C269D5310E09D68002D0AD119
:102040001D69002D03D1FF255C269D5306E07F25E9
:102050005C269D5302E025005C269D5384255C513F
:10206000222480255C51EFF31084012585F310882C
:102070001D68AD6801262E431D68AE6084F310888C
:102080009C68844205D11869002802D135489866B9
:1020900001E035489866186900280ED0EFF31080EB
:1020A000012484F310881C68246890256D00254362
:1020B0001C68256080F310880CE0EFF31080012489
:1020C00084F310881C682468202525431C6825603B
:1020D00080F31088002070BDFFFFFBFFFF7FFFFF34
:1020E000FFEFFFFFFFDFFFFFFFFFEFFFFFFF9FFFA0
:1020F000FFFFF7FFFFFFFF0100B5EFF310810122A3
:1021000082F3108802681268144B1340026813604F
:1021100081F31088EFF31081012282F310880268A6
:10212000926801239A4303689A6081F31088016ED4
:1021300001290CD1EFF31081012282F3108802688B
:10214000126810239A4303681A6081F310882021D3
:102150008022815000210166816600BDDFFEFFFF05
:10216000FF010000A1220008B321000838B50400D7
:10217000656A00205A21685252216852280000F0F6
:102180008DFA31BD10B50400EFF31080012181F309
:10219000108821680968402291432268116080F309
:1021A00010882020E0670020E066200000F0D0FDCD
:1021B00010BD70B504005C20255A802020582228CC
:1021C00067D12068808C0600300029000140606DD6
:1021D0000170606D401C60655A20205A401E5A21D3
:1021E00060525A20205A002859D1EFF31080012163
:1021F00081F3108821680968654A0A4021680A60ED
:1022000080F31088EFF31080012181F3108821689A
:102210008968012291432268916080F31088202010
:10222000802160500020A06660662168496809022C
:102230000CD5EFF31081012282F310882268126816
:10224000544B13402268136081F31088216E0129DA
:102250001BD12066EFF31080012181F310882168E3
:102260000968102291432268116080F310881020C1
:102270002168C9690140002901D0216808625820FD
:10228000215A200000F00BFA09E0200000F0C2FD06
:1022900005E020688069082101432068816170BDE4
:1022A000F8B504005C20255A80202058222867D1E8
:1022B0002068808C0600606D070028003040388060
:1022C000606D801C60655A20205A401E5A21605261
:1022D0005A20205A002859D1EFF31080012181F3B0
:1022E0001088216809682A4A0A4021680A6080F338
:1022F0001088EFF31080012181F31088216889682C
:10230000012291432268916080F31088202080216F
:1023100060500020A06660662168496809020CD5FB
:10232000EFF31081012282F3108822681368194AA2
:102330001A4023681A6081F31088216E01291BD18D
:102340002066EFF31080012181F31088216809686D
:10235000102291432268116080F3108810202168B8
:10236000C9690140002901D0216808625820215A1A
:10237000200000F094F909E0200000F04BFD05E09A
:10238000206880690821014320688161F1BD000057
:10239000DFFEFFFFFFFFFFFB70477047F8B504004B
:1023A00000252F00002C01D1012020E00220212156
:1023B0006054206801680E4808406168A2680A43BA
:1023C000E168114322690A4361691143A2690A4322
:1023D000E6691643064320680660200000F04BF9CA
:1023E000A563012021216054202025540020F2BD46
:1023F0000FC0FFFF38B50400002C01D1012021E0FF
:102400002068006801218843216808600025206851
:10241000056020684560206885602068C5602000F0
:1024200000F029F90120216C8840E16B4860A56229
:10243000E56225636563A56328002121605420209F
:102440002554002032BDF7B504001F00002006000F
:102450002021615C012901D1022039E001252900F8
:102460002022A1542121615C01292BD102212122AA
:10247000A154A06320680068012188432168086096
:102480003B00029A0199200000F0E0F8E06A002881
:1024900006D0206800680E210143206801600BE02F
:1024A000206800680A2101432068016020680068F4
:1024B000042188432168086020680068054320687B
:1024C000056003E020216054022006003000C0B205
:1024D000FEBD00B501002120085C022806D00420C2
:1024E0008863002020228854012017E008680068D3
:1024F0000E2290430A681060086800680122904329
:102500000A68106001200A6C03009340CA6B536094
:1025100021228854002020228854002000BD38B594
:102520000400002005002121615C022904D0042060
:10253000A063012005001BE0216809680E22914379
:1025400022681160216809680122914322681160A4
:102550000121226C0B009340E26B53602122A154B5
:1025600020216054606B002802D02000616B8847F6
:102570002800C0B232BD70B50400E06B0568206869
:1025800006680420216C02008A402A40002A16D0E6
:10259000064214D021680968890605D421680968B3
:1025A0000422914322681160216C8840E16B4860ED
:1025B000E06A002849D02000E16A884745E002200F
:1025C000216C02008A402A40002A1CD006421AD000
:1025D00021680968890608D4216809680A2291439C
:1025E0002268116001212122A154216C8840E16BF5
:1025F0004860002020216054A06A002825D02000D7
:10260000A16A884721E00820216C02008A402A4004
:10261000002A1AD03040002817D0206800680E2108
:102620008843216808600120216C02008A40E16B28
:102630004A60A06321216054002020216054206B57
:10264000002802D02000216B884770BD30B50124DE
:10265000056CAC40C56B6C60046863604468102C0A
:1026600004D10468A2600468E16003E00468A1602A
:102670000468E26030BD10B50400206805494018C8
:102680001421FEF71AFF800020640348E06310BDA8
:1026900000000000F8FFFDBF0000024070477047D7
:1026A000F8B584B00400002C01D101204AE2207862
:1026B000C00766D50C20B4490A680240042A09D034
:1026C0000A68104008280ED18020400209680140A5
:1026D000814208D1AD480068800352D56068002867
:1026E0004FD101202EE26068012806D1A748016879
:1026F000802252020A43026024E06068002809D167
:10270000A2480168A24A0A4002600168A14A0A4040
:10271000026017E0606805280BD19C4801688022A0
:10272000D2020A4302600168802252020A43026018
:1027300008E096480168964A0A4002600168954A96
:102740000A400260606800280DD000F0FBFA050026
:102750008E480068800314D400F0F4FA401B65280A
:10276000F6D30320EEE100F0EDFA0500874800689B
:10277000800306D500F0E6FA401B6528F6D3032057
:10278000E0E102262068304000284FD00C207E492E
:102790000A680240002A06D00A681040082814D1AE
:1027A0000868C00311D4794801683140002904D079
:1027B000E168012901D00120C4E10168F8229143B8
:1027C0002269D2000A43026030E0E06800281AD093
:1027D0006E4F386801210143396000F0B3FA0500FB
:1027E00038683040002806D100F0ACFA401B0328BE
:1027F000F6D30320A6E13868F82188432169C9008F
:102800000143396012E0614F386801218843386024
:1028100000F098FA050038683040002806D000F033
:1028200091FA401B0328F6D303208BE120780007A0
:1028300028D5E069002812D0C34F38680121014330
:10284000396000F07FFA050038683040002819D15F
:1028500000F078FA401B0328F6D3032072E1BA4F48
:10286000386801218843386000F06CFA0500386848
:102870003040002806D000F065FA401B0328F6D34C
:1028800003205FE1042720683840002800D18CE055
:1028900000206946087080204005AC490968014065
:1028A00000290AD1A9490A6802430A600968084058
:1028B00003900398012069460870A5480068C00588
:1028C00014D4A3480068802149000143A048016056
:1028D00000F038FA05009E480068C00506D400F0F4
:1028E00031FA401B6528F6D303202BE1A0680128AC
:1028F00005D19848016801220A43026021E0A068DE
:10290000002809D1934801680122914301600168C0
:1029100004229143016014E0A068052808D18D4885
:10292000016839430160016801220A43026008E03E
:1029300088480168012291430160016804229143A3
:102940000160A06800280FD000F0FCF90500814864
:102950000068304000281FD100F0F4F9401B7E4988
:102960008842F4D30320EDE000F0ECF9050079484B
:102970000068304000280FD000F0E4F9401B764991
:102980008842F4D30320DDE004100240001002402E
:10299000FFFFFEFFFFFFFBFF68460078012804D120
:1029A0006A4801686D4A0A4002602078C00650D526
:1029B0006069012822D1B44800680743B248076023
:1029C000B148006801210143AF48016000F0BAF945
:1029D0000500AD4800683040002806D100F0B2F98B
:1029E000401B0328F5D30320ACE0A7480168F82278
:1029F0009143A269D2000A4302602AE00421C9433C
:102A0000606988420BD1A0480268114001600168EA
:102A1000F8229143A269D2000A43026019E09A4861
:102A20000068074398480760974800680121884379
:102A30009549086000F086F9050093480068304029
:102A4000002806D000F07EF9401B0328F5D30320B0
:102A500078E0206A002874D08C4800680C2101407E
:102A600008294DD0206A022838D1894F3868894911
:102A70000140396000F066F900908026B60438689D
:102A80003040002807D000F05DF90099401A032873
:102A9000F3D3032056E09F4801680F229143E26A76
:102AA0000A430260794801687B4A0A40A16A1143DF
:102AB000626A0A4302603868802149040143396030
:102AC00000F040F9050038683040002839D100F0A6
:102AD00039F9401B0328F6D3032033E06C4E3068ED
:102AE0006C490140316000F02DF90500306880012B
:102AF00027D500F027F9401B0328F7D3032021E056
:102B0000206A012801D101201CE060480068019082
:102B10008048006802900198802149020840616A5B
:102B200088420CD102980007000FE16A884206D162
:102B30000198F02189030140A06A814201D001205F
:102B400000E0002005B0F0BD241002401C1002403F
:102B5000007000402010024089130000FFFFFFEFCB
:102B6000F3B581B00400002C01D101208BE00125D8
:102B7000694E30682840029988420CD230680121A1
:102B800088430299014331603068284002998842A5
:102B900001D0012077E002202168014000290FD0F8
:102BA0002178490705D539490A68E023DB0013433A
:102BB0000B6036490A68F0239A43A36813430B60FD
:102BC00021682940002932D06168012905D13048A7
:102BD0000068800311D4012055E06168022905D105
:102BE0002B480068800108D401204CE0284909687E
:102BF0000840002801D1012045E0244F3868032116
:102C0000884361680143396000F09CF8009038689F
:102C10000C21014060688000814208D000F092F8E9
:102C20000099401A3D498842F1D303202BE00298D5
:102C30003168294088420CD23068012188430299CA
:102C400001433160306805400298854201D001207F
:102C500019E02078400706D50C480168304A0A4040
:102C6000E1681143016000F019F82E49074A126823
:102C700012091207120F895CC8402B490860002016
:102C800000F0E6F80020FEBD3410024004100240BF
:102C900000100240FFFFFFFEFFFFC2FFF8B5002457
:102CA000200000942500260020490F680C2139409F
:102CB000042902D0082902D01BE01D481AE00F2089
:102CC0001C49BA0C0240895C0E001B49114A12686B
:102CD0001040085C0090F80306D515480099FEF7EF
:102CE000ECFB7043050002E0144870430500280027
:102CF00000E00F48F2BD0C480068704780B5FFF750
:102D0000FAFF0F49094A1268120A5207520F895CEA
:102D1000C84002BD2C100240002002408913000070
:102D2000FFF8FFFFB84C00085400002004100240D8
:102D300000127A00984C0008A84C000800093D00D9
:102D4000FC4C000801480068704700BF7804002070
:102D50007047FEE700B50200D205D20D364B1A804F
:102D6000364A1268D2695206FAD500BD38B586B027
:102D70008020800232490A6802430A6009680840DC
:102D8000009000988020C0012E490A6802430A6022
:102D900009680840009000980420019002200290E9
:102DA000012403940320049005949025ED0501A9C6
:102DB000280000F075F808200190059401A928006A
:102DC00000F06EF81D4C20482060E1204002606059
:102DD0000020A060E0602061A0610C216161606260
:102DE0002000FEF773FD2000FEF730FD00220221D7
:102DF0001B2000F0F6F91B2000F0FDF90122134919
:102E00002000FFF701F907B030BD80B50B48FEF791
:102E100080FD01BD10B504000C490878064A1080F9
:102E200006480268D2695206FAD50122FFF7ECF88B
:102E300000F03EFA10BD000028380140DC00002000
:102E40001410024018100240003801408F04002086
:102E500010B50400FA2080000E490978FEF72DFB1A
:102E600001000D480068FEF728FB00F0CBF90028B0
:102E700001D001200CE0042C09D200222100002006
:102E8000C04300F0AEF905480460002000E00120D6
:102E900010BD00BFD80000205400002050000020CA
:102EA000F1B582B000230868D840002800D1F3E0D3
:102EB0000124086825009D400540019501980028DF
:102EC00000D1E7E0032548682840012803D048687E
:102ED000284002281ED1029886681F00022047431E
:102EE0002800B8408643CF68BC46180002277843C4
:102EF00067468740374302988760029846682000FB
:102F000098408643486800092040984030430200BA
:102F10000298426048682840032812D00298C66888
:102F20001F00022047432800B84086438F68BC46F4
:102F30001800022778436746874037433A000298D3
:102F4000C26048682840022821D10298DE08042780
:102F50007E438019076A072000970F26B4461F009A
:102F60000740042677436646BE40009FB743BC46F1
:102F70000E691F00384004277843864067463E4369
:102F800032000298DE0804277E438019026202980C
:102F900006681F00022047432800B84086434F6858
:102FA0002F40BC46180002277843674687403743C6
:102FB0003A00029802604868C026B6020640002E19
:102FC00068D04948066826430660006820400090A3
:102FD0000098464E980804277843305800900F27F1
:102FE000BC461F00280038400427784367468740C6
:102FF0000098B843009002989027FF05B84201D18D
:10300000002410E002983A4A90420CD00298394AC3
:10301000904201D1022406E00298374A904201D141
:103020002C0000E0052400981A00154004225543A6
:10303000AC40044398080422504334502F4A10688F
:10304000019DA8434D68ED0202D50400019820437C
:1030500010602B4C2268019DAA434D68AD0202D539
:103060001000019A02432260264C2068019DA8436B
:103070004D68AD0302D50200019810432060224C38
:103080002268019DAA434D68ED0302D51000019A04
:10309000024322605B1C06E7F7BD00B50200106921
:1030A0000B009BB21840002801D0012000E0002056
:1030B000C0B200BD00B51300DBB2002B03D00B0083
:1030C0009BB2836102E00B009BB2836200BD10B42F
:1030D00042690B009BB213401B040C00A4B2944342
:1030E0001C43846110BC7047181002400800014066
:1030F0000004004800080048000C00480804014093
:103100000C040140040401400004014000B501002A
:1031100049B2002905D40121C206D20E91403C4A91
:10312000116000BDF0B5020052B2002A1CD4032287
:10313000384B040064B2A40804256C431C59FF25D5
:103140001600064008277E43B540AC438D01EDB222
:1031500002400826724395402543020052B292086D
:10316000042462439D5022E00F242B4A03230500D0
:103170006DB22540083DAD0804267543060076B2C1
:103180003440083CA408042674431659FF27BC4663
:103190001C00044008277C436746A740BE438C01BF
:1031A000E4B2034008277B439C4034435451F0BDB4
:1031B00010B50400601E80214904884201D301201B
:1031C0000EE0601E1549086003210020C043FFF790
:1031D000A9FF00201249086007201249086000205A
:1031E00010BD70B505000C0016002100280040B28B
:1031F000FFF798FF70BD10B50400200040B2FFF744
:1032000085FF10BD10B504002000FFF7D1FF10BDF1
:1032100000E100E000E400E01CED00E014E000E06C
:1032200018E000E010E000E038B5802080023A4964
:103230000A6802430A600A681040009000988020E3
:10324000C0020A6802430A600968084000900098BA
:10325000324D334828603348E860334868600024C2
:103260002C61AC606C61AC61280000F071F8002248
:1032700002211520FFF7B5FF1520FFF7BCFF28003E
:1032800000F094F829482A4901602A49C1602E4972
:103290004160046184604461846100F059F8002257
:1032A00002211620FFF79DFF1620FFF7A4FF31BD76
:1032B00080B52148008800F005FA00F013FA1FA23B
:1032C0000CCAFEF7B2F900221E4BFEF703F8FDF719
:1032D000CFFF1E49086001BD10B5040020681049E9
:1032E000884206D100F0B8FA002809D000F000FBAF
:1032F00006E020680E49884202D10C4800F083F8AD
:1033000010BD80B5054800F0A5F801BD80B507489F
:1033100000F0A0F801BD000018100240CC0200200F
:1033200000440140E70300007FBB000014030020BD
:1033300000480140CF07000088040020448B6CE760
:10334000FB69274000804740BF120000284401402D
:1033500010B50400002C01D1012026E03D20205CA6
:10336000002805D100203C216054200000F0A8F97D
:1033700002203D216054211D206800F05FF90120EA
:10338000462160543E2160543F21605440216054E6
:1033900041216054422160544321605444216054CF
:1033A000452160543D216054002010BD10B501003E
:1033B0003D20085C012801D0012023E002203D23AC
:1033C000C85401200B68DB6803430C68E3600B689A
:1033D0001E4CA34203D00B681D4CA3420CD10B68BA
:1033E0009B685B075B0F1A00062A0AD00B681B68F4
:1033F00018430B68186004E00B681B6818430B68DF
:103400001860002010BD00B501000868C0680122E6
:1034100090430A68D0600868006A0A4A0240002A9D
:103420000BD10868006A084A0240002A05D10868E2
:103430000068012290430A68106001203D228854F0
:10344000002000BD1111000044040000002C0140C8
:103450000004004070B50400022620680069304076
:1034600000281CD02068C0683040002817D00220F7
:10347000C0432168086101202077206880698007A7
:10348000800F002803D0200000F043FA05E0200060
:1034900000F09AFA200000F098FA00202077042526
:1034A00020680069284000281CD02068C068284097
:1034B000002817D00420C0432168086126772068BF
:1034C0008069C02189000140002903D0200000F05C
:1034D00020FA05E0200000F077FA200000F075FAED
:1034E00000202077082620680069304000281BD083
:1034F0002068C0683040002816D00820C0432168EA
:10350000086125772068C0698007800F002803D0F4
:10351000200000F0FEF905E0200000F055FA200040
:1035200000F053FA0020207710202168096901403B
:1035300000291CD02168C9680840002817D0102035
:10354000C0432168086126772068C069C0218900CE
:103550000140002903D0200000F0DBF905E0200045
:1035600000F032FA200000F030FA0020207701202D
:1035700021680969014000290BD02168C968084009
:10358000002806D00120C043216808612000FFF711
:10359000A3FE802021680969014000290BD0216821
:1035A000C9680840002806D08020C043216808610F
:1035B000200000F00BFA4020216809690140002931
:1035C0000BD02168C9680840002806D04020C043BD
:1035D00021680861200000F0FAF9202021680969BB
:1035E000014000290BD02168C9680840002806D096
:1035F0002020C04321680861200000F0E9F970BD77
:1036000000B5020000200B00002B06D0042B08D0D0
:10361000082B0AD00C2B0CD00FE013685B6B180042
:103620000BE013689B6B180007E01368DB6B180056
:1036300003E013681B6C1800FFE700BD10B50368BA
:10364000194A904202D0194CA04204D17024A343DD
:103650001C004B68234390420BD0144CA04208D06E
:10366000134CA04205D0134CA04202D0124CA042F1
:1036700003D1124C1C40CB6823438024A3434C69E4
:103680001C4304608B68C3620B688362904205D060
:10369000084A904202D0084A904201D10A69026366
:1036A0000122426110BD0000002C014000040040D6
:1036B000002000400044014000480140FFFCFFFFA3
:1036C0007047FEE79D2102000AD002D4491E9218DD
:1036D000FCD5C905100A1206524100D3012A4841FF
:1036E00070470000012212060118CA420AD28A421B
:1036F0000DD83822120609098918C20FD2071143C2
:103700004007704700D049080909014301E0C10F93
:10371000C90700207047FEE7F8B586B014220021E3
:1037200001A800F056F98020800246490A68024349
:103730000A6009680840009000981027019700244B
:10374000029401250395049401A99020C005FFF778
:10375000A7FB3D4E9020C0053060B7800220F0806E
:103760003A48F0603A483061B4612820B0832000C4
:10377000B077300000F04CF8B07240200190029415
:103780000395049401A99020C005FFF789FB07B0B9
:10379000F0BD704780B52C4800F001F801BD70B550
:1037A0000400E07A022814D0A1882068FFF775FC95
:1037B00006003000C0B2002802D10020E07201E013
:1037C0000120E072E07AA17A88421ED00220E072E5
:1037D0001BE02089401C2081E0882189884214D286
:1037E000002528002081A1882068FFF756FC0600EC
:1037F000A5613000C0B2002803D1E572206980477E
:1038000003E00120E072E0688047E07AA07270BDBA
:1038100010B50400A1882068FFF73FFC10BD80B5FB
:1038200000F01AF8002802D100F02AF905E0012280
:1038300020219020C005FFF73DFC064800F082F9EA
:1038400001BD000014100240380400201F38000899
:1038500093370008D84C000880B540219020C0055F
:10386000FFF71BFC002801D0012000E00020C0B2BF
:1038700002BDFEE738B586B01422002101A800F091
:10388000A8F8802080021E490A6802430A600A687C
:103890001040009000988020C0020A6802430A602D
:1038A0000968084000900098A02001900125029529
:1038B0000020039004909024E40501A92000FFF764
:1038C000EFFA01950F4D01A92800FFF7E9FA01224F
:1038D00001212800FFF7EEFB012220212000FFF745
:1038E000E9FB012280212000FFF7E4FB07B030BD97
:1038F00080B520219020C005FFF7E9FB01BD000045
:10390000141002400004004880B52748FFF7A2FDCC
:1039100001BD38B50400207F012841D1234D00218D
:103920002000FFF76DFE28602868002833D01D486E
:103930002968FDF7C2FD1F4908601D4D04212000C4
:10394000FFF75EFE286028681B4988420AD31B489F
:103950000178491C0170002204219020C005FFF766
:10396000A9FB0BE000200100154A117013490870F3
:10397000012204219020C005FFF79CFB0F4800782E
:1039800010280DD10E480178002909D101210170BC
:103990000C48017004E000200549086005490860F2
:1039A00031BD000040420F00840200206C04002062
:1039B0007004002074040020410600008D040020E3
:1039C0008C0400208B0400207047704770477047BC
:1039D000704710B50400080011000200200000F03C
:1039E000C5F8200010BDFEE770B586B01422002196
:1039F00001A8FFF7EEFF802080024E490A680243CB
:103A00000A600A681040009000988020C0020A688E
:103A100002430A6009680840009000980120029063
:103A2000022003900026049635000A2D17DA424C36
:103A30000820684320188088019001A90820684365
:103A40002058FFF72DFA00220820684320188188AB
:103A5000082068432058FFF72DFB6D1CE5E7300078
:103A60000A280BDA3549320004234343CA54320092
:103A700004234343C9184A80401CF1E706B070BDD7
:103A800038B52F4C2C48012221780823594341187E
:103A90008988237808256B43C058FFF70BFB01206A
:103AA0002649227804235A4388542078401C2070E9
:103AB00020780A2801D10020207031BD38B50025BA
:103AC0002C000A2C34DA1D4804216143415C012991
:103AD0002CD10421614341184988491C04226243C6
:103AE00082185180042161434118498832291DDB25
:103AF0002900042262438154290004226243801871
:103B000041800D480022082161434118898808231B
:103B10006343C058FFF7CEFAFFF79EFE002805D199
:103B2000002220219020C005FFF7C4FA641CC8E7DA
:103B300031BD0000141002400000002010040020DD
:103B40008A0400200EB4C0B5020003A80190002032
:103B5000009001AB0121044878440C30FCF7A8FA2E
:103B6000029906B0084700BFFB1000001206130AB6
:103B70001A43130C1A4300BF094205D0830705D02E
:103B80000270401C491EF9D1704700001300103923
:103B900006D330B41400150010393CC0FCD230BC40
:103BA000490700D30CC000D504C0890002D30280AD
:103BB000801C002900D502707047FEE7F8B50400AC
:103BC00000252F002E00002C01D10120D4E0A06B95
:103BD000002806D1E563280034216054200000F05D
:103BE000B5FB1020A16B0140002900D0BDE03900D9
:103BF000C9B2002900D0B8E00422216889681140C8
:103C0000002900D0B1E0A36BA349194002230B4364
:103C1000A363216889688907890F01290AD10121D5
:103C200023681B680B40002B03D12368DB681B044F
:103C300000D500E0290000290FD12168C9681823A8
:103C40009943A3680B432168CB60216809698B0005
:103C50009B0861681943236819612168CB688F4903
:103C600019402368D960A16A012902D08021490145
:103C700000E029002369022B00D02A00B446237EED
:103C80009E03637EDB033343A67E76031E433143EC
:103C9000E3680B431A432421615C4E0016436146DE
:103CA0000E43E17E01290FD1A17E002904D131000C
:103CB000802676020E4307E0A16B20220A43A2630E
:103CC000E16B01220A43E263E169FF22C2329142C1
:103CD00004D03200E169266A0E4316432168C968A0
:103CE00031432268D160E16A80225205914214D0AA
:103CF000E16A012911D0E16A02290ED0E16A0329A3
:103D00000BD0E16A042908D0E16A052905D0E16AEF
:103D1000062902D0E16A07290ED1216849690722E4
:103D2000914322685161216849692C22A25C5207A3
:103D3000520F0A4321684A612168C968584A0A40FB
:103D4000B24207D1E563A06B022188430121014300
:103D5000A1630FE0A16B022291430843A0630120FD
:103D6000E16B0143E163070004E0A16B0843A0633A
:103D7000012007003800C0B2F2BDF8B504000025EC
:103D80002F00002C01D101204EE0A06B0221014345
:103D9000A163200000F04DFA06003000C0B20028F8
:103DA00009D1200000F0F6F906003000C0B2012869
:103DB00001D00120A0633000C0B2012830D02068BB
:103DC00040689F218843216848609F2021680860DF
:103DD0002068C068334901402068C16020680069DC
:103DE00080008008216808612068406907218843B5
:103DF000216848612068006A2B49014020680162FF
:103E00002068806AC00CC004216888622748016865
:103E1000274A0A400260200000F099FAE563A56392
:103E2000342025543000C0B2F2BDF8B5040000259E
:103E30002F000426206880683040002826D13420D6
:103E4000205C012801D1022024E0012034216054AB
:103E5000607E012803D0200000F03AF90700380006
:103E6000C0B2002814D1A06B12490140802040004C
:103E70000843A063E563342025541C2021680860B2
:103E80002068806806432068866001E00220070001
:103E90003800C0B2F2BD0000FFFEFFFF1902FEFFB6
:103EA000E7FF3F8300023E8300F000F00827014057
:103EB000FFFF3FFFFEF1FFFFF7B5040000252800DC
:103EC000694608700427206880683840002844D17B
:103ED0003420205C012801D1022043E0012630007B
:103EE00034216054607E012804D0200000F0F0F8F6
:103EF0006946087068460078002831D1A06B1A49DD
:103F00000140802040000843A063E563342025542D
:103F10001648216B88621648216BC8621548216BD0
:103F200008631C2021680860206840681021014354
:103F3000206841602068C06806432068C660029B14
:103F4000019A206801004031206BFEF77CFA20685E
:103F5000806807432068876002E002206946087095
:103F600068460078FEBD0000FEF1FFFF9F4200089A
:103F7000214300082F430008F8B504000D00002776
:103F80003E00009780214905E06A884213D0E06A2C
:103F9000012810D0E06A02280DD0E06A03280AD078
:103FA000E06A042807D0E06A052804D0E06A062801
:103FB00001D0E06A07283420205C012801D10220CA
:103FC00085E0012210003423E05420688068400717
:103FD00074D468686B4B984256D02068806A2B680E
:103FE0009A40024320688262E06A884228D0E06AF0
:103FF000012825D0E06A022822D0E06A03281FD0D9
:10400000E06A04281CD0E06A052819D0E06A062876
:1040100016D0E06A072813D00720A96822685269E1
:10402000024091420CD021684969072291432268DD
:10403000516121684969AA681040084321684861B4
:104040002868102802D0286811283CD12868102838
:1040500002D18020000401E08020C0034A490A68A0
:1040600010430860286810282DD148480068484946
:10407000FDF723FA0A21484300900098002822D037
:104080000098401E0090F8E72068806A29688A40FE
:104090009043216888622868102802D02868112877
:1040A00011D12868102802D18021090401E0802163
:1040B000C903354802688A43026004E0A06B2021EE
:1040C0000143A1631600342027543000C0B2F2BD72
:1040D0007CB50400002006000090216889688907EB
:1040E000890F01290BD10121226812680A40002A98
:1040F00003D12268D268120401D50800FFE7002826
:104100003DD12068806884490140002909D0A06B16
:1041100010210143A163E06B01210143E163012010
:104120002EE00125206880682843216888601748B0
:1041300000681749FDF7C1F900900098002803D0E6
:104140000098401E0090F8E7FEF7FCFD060020688E
:1041500000682840002812D1FEF7F4FD801B0328D8
:10416000F5D32068006828400028F0D1A06B10210A
:104170000143A163E06B0543E563012000E00020FB
:1041800076BD000001100000082701405400002007
:1041900040420F0070B50400002005000321226892
:1041A00092680A40012A0BD1012223681B68134040
:1041B000002B03D12368DB681B0401D51000FFE747
:1041C000002834D02068806805220240012A0BD1E3
:1041D00020688068022202432068826020680160B3
:1041E000FEF7B0FD050009E0A06B10210143A163BB
:1041F000E06B01210143E163012019E00126206801
:1042000080683040002812D0FEF79CFD401B032838
:10421000F4D32068806830400028EFD0A06B1021D4
:104220000143A163E06B0643E663012000E0002048
:1042300070BD70B5040000250426206880683040F9
:1042400000282AD0206880683040002809D02068E3
:104250008068800705D420688068102101432068A9
:104260008160FEF76FFD05002068806830400028FF
:1042700013D0FEF767FD401B0328F5D32068806844
:1042800030400028F0D0A06B10210143A163E06B07
:1042900001210143E163012000E0002070BD38B539
:1042A0000400656AA86B5021014000292FD1A86B3A
:1042B000802189000143A9632868C068C0210901E1
:1042C000014000291FD1A87E00281CD12868006861
:1042D000000718D52868806840070CD42868406813
:1042E0000C21884329684860A86B0C4901400120D3
:1042F0000843A86307E0A86B20210143A963E86B8A
:1043000001210143E963280000F017F903E02000D0
:10431000296B096B884731BD17000080FFFEFFFF46
:1043200038B50400656A280000F03EF931BD38B5A3
:104330000400656AA86B40210143A963E86B04216E
:104340000143E963280000F030F931BD7047704740
:10435000F8B586B01422002101A8FFF73AFB8020AF
:10436000800286490A6802430A6009680840009092
:104370000098802080007E490A6802430A6009682C
:1043800008400090009803270197029700240394A7
:1043900001A99020C005FEF783FD764D7648286080
:1043A0002800FFF7EAFC8020C0056860AC60EC6084
:1043B00001262E610420686120006876200028769E
:1043C0002000A8763000E876FF20C230E8612C6239
:1043D000300024216854AC62EF622800FFF7EEFB46
:1043E0006F4F3C6080204001786039002800FFF763
:1043F000C3FD3E6039002800FFF7BEFD280000F035
:10440000D5F8280000F002F807B0F0BD38B5040078
:1044100001205A490A6802430A600968084000906E
:104420000098574D5F48286000206860A860802091
:10443000E8608020400028618020C0006861202062
:10444000A86180208001E8612800FDF7D3FF2800E3
:10445000FDF7A4FF25636C62002201210920FEF70D
:10446000C0FE0920FEF7C7FE31BD38B504000D00BF
:104470002079142801DB002020716079142802DAE9
:104480006079401C607120682179042251436118D1
:10449000896800F031F920602068290000F0F4F804
:1044A000206020790100491C2171C0B204214843D9
:1044B000201885606079FFF705F90100206800F099
:1044C00073F932BD10B502000C001079142801DB1D
:1044D000002010715079142802DA5079401C507174
:1044E00010681179022359435118C988401A106085
:1044F0001068210089B24018106010790100491C31
:104500001171C0B2022148431018C480106851795B
:10451000FCF7D3FF80B210BD10B5164C02221B4928
:104520002000FFF7C9FC2000FFF77FFC10BD80B51D
:104530001048006BFEF71FF801BD38B50500134C9D
:104540002088FCF7ADFE12A20CCAFDF76EF800F051
:1045500080F901001048FFF788FF0B490860618867
:104560000E48FFF7AFFF07490880FEF7A1FE31BDF7
:1045700018100240A0030020002401401410024043
:104580005C030020880400206404002068040020EC
:10459000F564FED137694A3FDC010020E0030020CA
:1045A000580400200800024070477047FEB5040020
:1045B00000252F00019500953420205C012801D1B1
:1045C00002205EE00126300034216054032021687F
:1045D0008968014001290AD1216809683140002910
:1045E00003D12168C968090401D5310000E0290020
:1045F00000293DD1A16B234A0A4002211143A16346
:104600002168C968084000902068C0680321884379
:104610002168C860206880688021090601432068FD
:104620008160FEF78FFB019020688068002813D519
:10463000FEF788FB0199401A0328F5D320688068AB
:104640000028F1D5A06B0221884310210143A1630A
:1046500034202554012014E02068C06800990143EB
:104660002068C160A06B022188430643A66304E072
:10467000A06B20210143A16337003420255438006A
:10468000C0B2FEBDFFFEFFFF0122D20703004B4078
:104690002ED4431A01D2C01AC91830B44B180418CA
:1046A000240E1B0E22D0FF2C20D0E31A182B1DDC69
:1046B00009021143C40D641E0002104394461925DB
:1046C000ED1A0A00AA40D940451801D36D08A41C70
:1046D000E405D209280A2D062A436546AA4160410D
:1046E00003181B0EFF2B01D3C00DC00530BC704753
:1046F000514006E05140CCE70122D20703004B4075
:10470000F8D4431A03D2C01AC9185040514030B4EB
:104710004B18090211430418240E1B0E40D0FF2C25
:104720003AD025009D410BD31ED8C50D4002401A3A
:104730000BD3ED050100400AC90591416841D5E759
:10474000C50D40024918401AD0D001214008491C2B
:104750000018FCD58C4204D36D1A000AED054019EF
:10476000C4E7E8051040C1E7182DBFDCAC1C0D0004
:10477000E140E5414D40012D4941C40D0002104387
:10478000451A01D46D199543641EE405280A2D06C7
:104790009541604130BC7047FF2BA7D1D843A5E7B6
:1047A0002442A3D10020A1E730B405004D400122EE
:1047B000D20715404B180418240E28D01B0E2FD0FA
:1047C000FF2C34D0FF2B37D0E41A0002090210432B
:1047D000114343084808D10D1B1A02D2641EDB188E
:1047E0001B18DB18834200D31B1A4941F9D37F34CD
:1047F00026DDFE2C08DAE4054808C9071943914173
:104800006041284330BC7047FF20C005F9E728000D
:104810001B0E03D0FF2BF5D14902F3D0D043F1E7B3
:10482000FF2C01D14002F9D1FF20C005E9E7400289
:10483000F4D1FF2BF8D1F1E728004902E2D0EDE7EF
:104840000B0200202442DCD15B129B1CD9D9D80575
:10485000D7E7012252054B18DA4201D958157047A3
:104860005B0D0722D2019B1A10D9FF2B1DD2DB054D
:104870000122D2070A4013430903020D1143490ADA
:10488000C200524100D9491CC81870470AD1800A99
:104890000A0302435212921C04D9D3070B40D005DD
:1048A00018437047C80FC0077047C80F0002FF3099
:1048B000C005704780B500F089F800F075F83F48F2
:1048C0000178491C017001780A2901D10021017089
:1048D00000200A2824DA3A490C2242438A18127A24
:1048E000002A1BD00C2242438A189288521E0C23A5
:1048F0004343CB189A800C2242438A189288002A9C
:104900000CD10C2242438A18D2880C234343CB1883
:104910009A8001220C234343C9184A72401CD8E7ED
:1049200001BD70B500231A000A2A24DA244C0C2594
:1049300055436559002D1CD101250C265643A61957
:1049400035720C25554365196B720C235343E150A6
:104950000C235343E318D8800C235343E318DB881C
:104960000C2555436419A380164B1C68641C1C60FD
:1049700001E0521CD8E770BD38B5002425000A2D8F
:1049800011DA0F480C2169434118497A002908D0EF
:1049900021000C226A43821851720C21694340584D
:1049A00080476D1CEBE731BD00B507480168002961
:1049B00002D00168491E016000BD00008E04002085
:1049C00064010020800400207C040020034801686A
:1049D000034A127889180160704700BF78040020EC
:1049E000D800002080B500F063F800F02BF8FEF747
:1049F000FBFFFEF73FFFFFF7ABFCFEF715FCFEF7F2
:104A00008BFEFEF7B3F90B48FFF79CF8FA20800005
:104A100000F060F808490A20FFF783FF07490A20E1
:104A2000FFF77FFF06490A20FFF77BFFFFF7A4FF90
:104A3000FCE70000884C000819450008953700087D
:104A4000BD3A000838B590B03022002104A8FEF726
:104A5000C0FF102200216846FEF7BBFF1220049021
:104A6000012007900990102008900A9002240C94CD
:104A700000250D95A02080030E900F9504A8FDF74A
:104A80000FFE002801D000F00FF8072000900194DD
:104A90000295039501216846FEF762F8002801D0CF
:104AA00000F002F811B030BD00B572B6FEE7FEE7C7
:104AB00080B50648016810220A4302600020FEF714
:104AC000C7F900F005F8002002BD000000200240F8
:104AD0007047FEE770B50400FEF734F905002600C4
:104AE0000020C043864202D0044800783618FEF702
:104AF00029F9401BB042FAD370BD00BFD800002096
:104B0000686A6C747A4C00007072696E74665F73C8
:104B10003A20256E20646973616C6C6F7765640060
:104B20007072696E74663A2062616420256E20613D
:104B30007267756D656E74007072696E74665F730E
:104B40003A2062616420257320617267756D656E1D
:104B500074000000000000006E616E004E414E00C7
:104B6000696E6600494E4600300070B4012300248F
:104B700013E00168001D194202D04D466D1E49190F
:104B80000C60091D121F042AFAD20D00960701D5E8
:104B90000C80AD1C1A4000D02C700268001D002A49
:104BA000E7D170BC704730B50168411844686208AD
:104BB0008A188368E40704D54C461B1901E0641C7D
:104BC00006D191420BD00C7864B2491C0D78491C77
:104BD0001D705B1C002CF2D4641EF7D5F1E70C307D
:104BE00030BD000010B5074979441831064C7C44AB
:104BF000163404E0081D0A68891888470100A1429C
:104C0000F8D110BD08000000240000005FFFFFFF86
:104C1000B4030000DC000020000000008BFFFFFF59
:104C2000E60000004A0100000000002000F00DF83E
:104C3000002801D0FFF7D6FF00BF00BF002000BF53
:104C400000BFFFF7CFFE00F002F80120704780B5EB
:104C500000F002F801BD000007463846FCF7ECFD05
:104C6000FBE738B505000C00200000F005F8A04275
:104C700000D00025280032BD80B50249FEF76AF851
:104C800002BD00BF9000002046572073746172740B
:104C900065642E2E2E0D0A0002030405060708097E
:104CA0000A0B0C0D0E0F1010010203040506070875
:104CB000090A0B0C0D0E0F10000000000000000090
:104CC000010203040607080901488047014800471C
:104CD000054D0008F14C0008427574746F6E0D0AA2
:104CE0000000000000B5FEE700B5FEE77047704722
:104CF00000BF00BF00BF00BFFFF798FF000000002B
:104D0000010203047047FD0002480002FB00024854
:104D10000004FB0002480008FB0002480010FB00F2
:104D200002480080FD000304004880FC00030400EA
:104D30004840FC000304004820FC00030400481025
:104D4000FC000304004808FD000004FC001E127A69
:104D500000E24B0008E24B0008E24B0008E24B0087
:104D600008E24B0008E24B0008E24B0008F8FF0B9A
:104D700026110008E24B0008E24B0008FAFF15007C
:104D800000020401013402002084020020340200E9
:104D90002034020020FC000334020020FC0007D471
:0B4DA000000020C0000020E000000127
:0400000508004CF1B2
:00000001FF
